:020000040000FA
:0400000046EF00F0D7
:020008002AD0FC
:08001800D8CF01F0E8CF00F0A1
:10002000E0CF02F0F6CF17F0F7CF18F0F8CF19F0C5
:10003000F5CF1CF09EB209EC05F0F2B43BEC0EF0EB
:1000400002C0E0FF00C0E8FF01C0D8FF17C0F6FF04
:1000500018C0F7FF19C0F8FF1CC0F5FF1000F6CF5D
:1000600014F0F7CF15F0F8CF16F0F5CF1BF0A1B2D2
:1000700080ED03F09EB091ED03F014C0F6FF15C0C3
:10008000F7FF16C0F8FF1BC0F5FF1100C26AEF0EA4
:10009000C16E070EB46E000E926EFF0E936E000ED0
:1000A000946E700ED36E400E9B6E00EE00F000EC6E
:1000B0000FF0D08E899E27822798279A279694EC56
:1000C00002F080EC02F08AEC02F000EC05F035EC76
:1000D0000EF000EC0EF027826CEF00F081B076EFAE
:1000E00000F081B27EEF00F06EEF00F0278881B261
:1000F0007EEF00F081A4278676EF00F0278A6EEF6E
:1001000000F081EF00F0000E106E100E0F6E000E6A
:0C011000F86ED6EC02F027928CEF00F0A5
:10050000B00EB16EF28CF28EA082A282B36AB26A91
:10051000B1801200B00ECD6EF28CF28E9D809F8065
:10052000CF6ACE6ACD8012000A0E216E276A0D9026
:10053000899E1200000EF66E100EF76E000EF86E19
:100540000900F552D8B4D5EF02F0BF0EF524206EA5
:100550000900D00EF526F8CF0EF0F7CF0FF0F6CF4A
:1005600010F0F5CF1AF02050070FF52EB4EF02F07F
:10057000F90F2050F66E180EF76E0800F5CF0CF04C
:10058000190EF76E0800F5CF0BF00D8088EC04F023
:100590000D909EEC04F00EC0F8FF0FC0F7FF10C0E6
:1005A000F6FF1AC0F5FFA0EF02F0120010C0F6FF30
:1005B0000FC0F7FF0EC0F8FF010E226E12EC03F021
:1005C000F8CF0EF0F6CF10F0F7CF0FF0F5CF1AF00E
:1005D000C60FD8B0FAEF02F01D0FD8B0F6EF02F058
:1005E000222A222A222A1D0FFBEF02F0222A1D0FA7
:1005F000FBEF02F03A0FEC0FF66E1A0EF76E000EDC
:10060000F86E0800F5CF23F01B0EF76E000EF86EA3
:100610000800F5CF24F00EC0F8FF10C0F6FF0FC0A1
:10062000F7FF12000900F55012000900F552D8B486
:100630003BEF03F0F652D8B4F72AF546F536D8B0BA
:1006400012002146F536D8B012002146F536D8B052
:1006500012002146F536D8B012002146F536D8B042
:1006600012002146F536D8B012002146F536D8B032
:0E067000120021461200278212001AEF03F03A
:10070000A1920C52D8B48CEF03F00CC0B3FF0BC015
:10071000B2FF0DB0897E12000C52D8B4120085EFE2
:1007200003F09E9027B204EF04F00EC0F8FF0FC054
:10073000F7FF10C0F6FF1AC0F5FF212EF7EF03F008
:1007400027B0EEEF03F022C021F00900F652D8B432
:10075000F72AF552D8B4ECEF03F0BF0EF524206E63
:100760000900F652D8B4F72AF552D8B4ECEF03F0EA
:10077000D00EF526F8CF0EF0F7CF0FF0F6CF10F031
:10078000F5CF1AF02050070FF52EC3EF03F0F90F45
:10079000F66E180EF76E0800F5CF0CF0190EF76E16
:1007A0000800F5CF0BF00EC0F8FF0FC0F7FF10C028
:1007B000F6FF1AC0F5FF15EC03F00D80278023C06B
:1007C000CFFF24C0CEFFF8CF0EF0F7CF0FF0F6CF5B
:1007D00010F0F5CF1AF0120027821200020E216EDF
:1007E0000D90A00ECF6E000ECE6E2790120027A0A7
:1007F000FFEF03F023C0CFFF24C0CEFF1200A00EF6
:0C080000CF6E000ECE6E12000D901200A4
:100900000400056E88EC04F0052E82EF04F012005E
:10091000640E066E550E076E060E086E040000008B
:100920000000000000000000082E8EEF04F0072EEB
:100930008CEF04F0062E8AEF04F012001E0E036EF8
:10094000140E046E0400000000000000000000000F
:100950000000042EA2EF04F0032EA0EF04F012001A
:10096000C80E096EC80E0A6E0A2EB4EF04F0092EE6
:10097000B2EF04F01200FF0E096E0000000000004C
:10098000092EBDEF04F01200096EC80E0A6E0A2E81
:0C099000C7EF04F0092EC5EF04F01200C0
:100A0000000ECA6EF28CF28E9D829F92CC6ACA84CE
:100A100012009E923D2E0FEF05F0640E3D6E3D508C
:100A2000296016EF05F089901AEF05F03AB0898039
:100A30003AA089903D502A6021EF05F0899225EF78
:100A400005F03AB289823AA289923D502B602CEF90
:100A500005F0899430EF05F03AB489843AA489947A
:100A60003D502C6037EF05F089963BEF05F03AB624
:100A700089863AA689963D502D6042EF05F0899A05
:100A800046EF05F03AB8898A3AA8899A3D502E6017
:100A90004DEF05F0899C51EF05F03ABA898C3AAADE
:100AA000899C3D502F6058EF05F08B905CEF05F06E
:100AB0003ABC8B803AAC8B903D50306063EF05F0D0
:100AC0008B9267EF05F03ABE8B823AAE8B923D5027
:100AD00031606EEF05F08B9472EF05F03BB08B84C4
:100AE0003BA08B943D50326079EF05F08B967DEF03
:100AF00005F03BB28B863BA28B963D50336084EF72
:100B000005F0899888EF05F03BB489883BA4899863
:100B10003D5034608FEF05F08B9C93EF05F03BB6B2
:100B20008B8C3BA68B9C3D5035609AEF05F08B9AE1
:100B30009EEF05F03BB88B8A3BA88B9A3D50366000
:100B4000A5EF05F08B98A9EF05F03BBA8B883BAA7F
:100B50008B983D503760B0EF05F08B9EB4EF05F0F9
:0A0B60003BBC8B8E3BAC8B9E120059
:101000005643320845320843320845320847320415
:101010004732044332084532084332084532084714
:10102000320447320443330842330841330847321D
:101030000846320441330447320846320845320834
:1010400044320843320443320441340243320445FB
:1010500032044332044532044732044732044332F7
:101060000445320443320445320447320447320413
:1010700043330442330441330447320446320441CB
:1010800033044732044632044532044432044332C6
:08109000044332044134010065
:10110000564332044731044332024532024432042A
:10111000433204443202443202433204473104432E
:101120003202453202443204433204443202443231
:101130000245320446320447320243320246320448
:1011400045320444320244320245320446320447F6
:1011500032024332024632044532044432024432FF
:0211600002008B
:101200005643320847310843320445320444320819
:10121000433208443204443204433208473108431D
:101220003204453204443208433208443204443222
:101230000445320846320847320443320446320835
:1012400045320844320444320445320846320847E5
:1012500032044332044532084432084332044332F4
:02126000040088
:101300005641330441330441330841330844320425
:10131000473204473204473208473208463204460F
:101320003208473208413308413308413308473215
:101330000841330844320847320446320445320833
:081340004532084432040000AC
:101500005641340441330446320446320447320221
:10151000473204473204413404473204453204431D
:10152000320444320244320444320441340441332C
:10153000044632044632044732024732044732043A
:1015400041340447320445320443320444320244F5
:1015500032044432044134044732044732044732EF
:101560000446320246320446320441340445320411
:1015700045320445320444320244320444320441C8
:1015800034044732044732044732044632024632BA
:1015900004463204413404453204453204453204E1
:1015A0004432024432044432040056413104423190
:1015B00004433104443104453104463104473104C5
:0215C000000029
:10180000F7F8F8F9FAFAFBFBFCFCFCFDFDFDFDFE28
:10181000FEFEFEFEFE0000000000000000000000D2
:0418200000000000C4
:101900001F178B5B1467048F0B43AC093382C70529
:101910002256849AC1000000000000000000000070
:0419200000000000C3
:101A000048515960676D73787D030B131B22282E94
:101A1000343A3F44484D5155595D6064676A6D7072
:101A20007375787A7D7F03070B0F13171B1E222512
:101A3000282B2E3134373A3C3F414446484B4D4FDA
:101A400051535557595B5D5F6062646567686A6CA6
:101A50006D6E70717374757778797A7C7D7E7F8016
:101A60008182838485868788898A8B8C8D8E8F90EE
:101A70009191929394959596979898999A9A9B9C00
:101A80009D9D9E9E9FA0A0A1A2A2A3A3A4A5A5A642
:101A9000A6A7A7A8A8A9A9AAAAABABACACADADAEA6
:101AA000AEAFAFAFB0B0B1B1B2B2B2B3B3B4B4B421
:101AB000B5B5B6B6B6B7B7B7B8B8B8B9B9B9BABAAE
:101AC000BABBBBBBBCBCBCBDBDBDBEBEBEBEBFBF4A
:081AD000BFC0C0C0C0C1C1C10C
:101B0000E59D8AC76984265D3570DCBC1E0D94BCDA
:101B10008C0C4133E55C9DAB8A3DC72A69868463A2
:101B200026CE5DD5358170B8DCDCBC7C1EA30D5D96
:101B300094B4BCAF8C560CB041C23393E5275C83A0
:101B40009DAAABA08A693D07C77D2ACE69FC86099C
:101B500084F763C8267DCE195D9CD508355E819FCC
:101B6000B8CCDCE7EEF0EEE8DED0BEA88F72512EE6
:101B700006DCAE7E4A13DA9D5E1CD79046F9AB595F
:101B800006B058FDA042E17E19B249DF72049321EC
:101B9000AE38C148CE52D556D553D04BC53DB42AE8
:101BA0009E1183F463D13EAA157EE74EB4197EE1FF
:101BB00043A40463C21F7BD7318BE43C93E93E937B
:101BC000E73A8CDE2E7ECE1C6AB7044F9AE52F785A
:081BD000C0084F96DC2166AA53
:101C00003A6A3B6A8B6A800E89161200010E296EB1
:101C1000020E2A6E030E2B6E040E2C6E050E2D6E18
:101C2000060E2E6E070E2F6E080E306E090E316EE8
:101C30000A0E326E1E0E336E320E346E460E356E46
:101C40005A0E366E640E376EFF0E3A6E3B6E120001
:101C5000296A3A80292A650E2918D8B4296AB0EC75
:101C600004F0B0EC04F02AEF0EF0070ED56EF194FC
:101C7000F28AD58E1200F29445EC0EF081B84AEC4F
:101C80000EF081BA6BEC0EF01200E70ED76E960ED6
:101C9000D66E12003BA25CEF0EF037C038F036C0B3
:101CA00037F035C036F034C035F033C034F032C0D0
:101CB00033F038C032F01200640E326E020E336E12
:101CC000346E356E366E376E3B823B843B863B8886
:101CD0003B8A3B8C12003AA083EF0EF031C039F002
:101CE00030C031F02FC030F02EC02FF02DC02EF0BC
:101CF0002CC02DF02BC02CF02AC02BF029C02AF0CC
:101D000039C029F01200640E296E020E2A6E2B6E65
:101D10002C6E2D6E2E6E2F6E306E316E3A803A82A2
:101D20003A843A863A883A8A3A8C3A8E3B80120054
:021D300012009F
:0C1E00000400EE6AEAA400EF0FF01200EC
:020000040030CA
:0100010008F6
:0100020010ED
:010003001EDE
:010005008179
:010006008178
:010008000FE8
:01000900C036
:01000A000FE6
:01000B00E014
:01000C000FE4
:01000D0040B2
:00000001FF
